:1074000080E189BD82E189BD09B400FEFDCF089508
:10741000CED569F08091E9008F931092E900A3D452
:1074200083FF01C022D58F9187708093E900089572
:107430008EEF0090E10008220092E1000895F20131
:10744000F999FECFF2BDE1BD0895F9DFF89A80B554
:1074500008C0F5DF1FBA80BD0FB6F894FA9AF99A02
:107460000FBE31962F010895E0E0F0E085919491F0
:10747000019608958AE28BB98BEA34D01092890084
:107480008AEF8093880082E080936F0083E080938E
:107490008100EDE5F7E785913AD0E936E1F781E043
:1074A0008093D7008AE482BF1092D8001092E20045
:1074B0001092DA001092E10080E808D019BC1EBAE0
:1074C0001092E00066D489E057D481E98093D80017
:1074D0000895A3E6B1E090E81AD08D939A95E1F76C
:1074E000089586E008D010C083E005D08F2F0FD01C
:1074F0008E2F0DD080E05B9A5A9809C005D085E0A8
:10750000FADF05D080FDFDCF5A9A5B9808958EBDB5
:107510008DB587FFFDCF8EB508958FE08221E9F705
:10752000F3DFE3E6F6E090EB5C98892FF0DF80E193
:10753000EEDF5C9A8191EBDF83E68E278F77D1F7C0
:107540009395983B89F708952E9858982D98E3E6DF
:10755000F1E094FC36C097FC4DC092FE08959684ED
:107560009920D1F3F894C089D78520E030E080E0FD
:1075700090E4AFEFBFEF119689199040E0F72D012D
:10758000BD4F8D0127FD13C0E0E0F8E011928EE7BA
:10759000819392E4E11791939AE508F092E4E33441
:1075A000C9F781931082BCDFFE0121969DDF91DF38
:1075B000F90100D520583F4F040D151D9A9411F77D
:1075C0000FC28301282D60906C0170906B0143D035
:1075D00019F48823C1F70895380188243CD0C9F5EF
:1075E00080916A01821709F4830160906E017090A6
:1075F0006D01F4CF80E8982E60906E0170906D015F
:107600002AD059F48823B1F708959FEF96FC03C060
:1076100095FE089591E097FB890E662477248301F7
:10762000222719D0B1F48823A1F380916A0136F0A2
:10763000881650F4821730F0213003C0881520F4EA
:10764000281710F48301282F60906E0170906D014F
:10765000E8CF3801822EF30147DF3BDFC3E6D1E0FC
:10766000E6E5F7E709908591081621F4ED35D1F7A5
:107670000880801049CFC9E02EDFCA95E9F7D0E134
:1076800094FC55C097FC37C095FE1AC0C3E6D2E003
:10769000E3E6F6E098E088E78E0F00840192E817B1
:1076A000E1F7884F09900192E817E1F7C858DF4FDA
:1076B0009A9589F732DFC85FD340C33E49F749C086
:1076C000C3E6D6E0EBE5FAE098E08E2F885702900B
:1076D0000086E817E1F738960A900292E817E1F77A
:1076E0003897C857D0409A9581F717DFC850DC4FBC
:1076F000C33E41F72EC0A3EEB6E0E3E6F6E09AE023
:10770000C6E00D9080818025807F802582958193C1
:10771000A336B90709F4B2E0E336F90709F4F2E059
:10772000E336FC0771F7F9DEDA9529F712C0A3EE0C
:10773000B9E0E3E6FAE092E00E90829180258F7046
:10774000802582958083E336F907B1F7E6DEDA9586
:1077500071F78827089541524455424F59D5F08D0D
:1077600014A1C881CFD9F1AF000000FFFFCFCFFF38
:10777000FFFFFFCFCFFFFF0000FE067E7E06FE4626
:10778000565616FE0656461EFE3F61E9E3FFE3EB42
:0A779000E3FFE3EBE3FFE16B3F00D2
:10779A001201100102000008412336000100000016
:1077AA00000109023E0002010080320904000001C2
:1077BA000202010005240010010424020405240623
:1077CA000001070582030800FF09040100020A00FC
:1077DA0000000705040210000107058302100001DA
:1078000011241FBE04B714BE88E18093600010925B
:1078100060008EEF9AE09EBF8DBF222433242101A9
:107820003101410180E88AC00F928F939F931F928C
:107830000FB60F9211244F936F938091DA0080FF5F
:1078400037C023C00F920FB68F939F93EF93FF9390
:1078500088278093850080938400E0E5F1E09281A1
:10786000907261F490818917980B908309F45D9A66
:1078700091818917980B918309F4289A239411F424
:107880008315381EFF91EF9154C08091D80080FF7E
:107890000FC08091DA008E7F8093DA008091D9004A
:1078A00080FF04C0ADDD81E08EBB02C019BC1EBAF2
:1078B0008091E10080FF0BC059D280FF08C059D2EF
:1078C0008091D800806202DE19BC85E08EBB809179
:1078D000E10084FF1AC04AD284FF17C091DD809175
:1078E000D8008F7DF3DD8FEEA4DD40D28F7E8160E6
:1078F00043D280915301882331F48091E30087FDC6
:1079000002C081E001C084E08EBB8091E10083FF72
:107910000CC02CD283FF09C087EF8BDD82E08EBBC9
:107920001092530185DD25D234D26F914F910F9083
:107930001F909F918F910FBE0F90189580936100BB
:1079400010926100B1E0B5BF82E085BF81E985B9E1
:1079500087EE84B91DB8769A10BA83EF81BB8CE2AA
:107960008BB98FE38AB980E58CBDBDBDA0E0EAE9A3
:10797000F7E705900D92A035E1F71D92BB30E9F7CE
:1079800001FD06C000FF04C07F9B02C06DDD41F514
:1079900071DD789460DE71F0ABE9B7E0E9E6F7E716
:1079A00090E105900D929A95E1F7A059BF4FE93902
:1079B000B9F7B7DD4FD02CDD80915201807861F4AA
:1079C0008FB18095807F66991C9B8460982E1DDE08
:1079D0008110BADD92FC02C0332062F745DD51F31D
:1079E000F89489EB7FDD81E08093E00010926F00D6
:1079F00010928100109285001092840081E085BF72
:107A000015BE5D9A289A0C940000ABD107C05ED1D8
:107A100002C0CDD239F0A7D182FFFBCF85FFF7CFCF
:107A20008091F1000895082E83E09CD185FD07C068
:107A300091D102C0BCD269F096D180FFFBCF0092F9
:107A4000F10080915201807221F45D9884E6809368
:107A50005001089586D182FF3BC18091520180720E
:107A600021F4289884E680935101CFDF182F8534C4
:107A700031F422248EE7382EE2DC8DE012C1843509
:107A800011F4C3DFFACF8C34C1F38035B1F38437FE
:107A900021F484E4C8DF80E004C1813611F489E573
:107AA00000C1813429F4B1DF582EAFDF482EE5CF75
:107AB000803711F483E5F5C0833539F4E6E5F7E75F
:107AC0008591B1DFED35E1F7EDC0863521F481E335
:107AD000AADF89E3E6C0863781F481E3669B8E5F87
:107AE0001C9B8F5FA0DF81E47C9B885F7D9B8C5F0C
:107AF0007E9B8E5F7F9B8F5FD4C08837C1F485DF0C
:107B000080935201289A84FD28985D9A83FD5D98A0
:107B100087FD8824877009F487602E9A81FD2E984E
:107B2000589A82FD58982D9A80FD2D98A6CF8A36B6
:107B300049F48FE9E0DCC3E0EADC75DFCA95E1F7E0
:107B4000E3DCB0C0833731F487E86DDF85E96BDFB4
:107B50008EE1A7C0853639F4E0E8F3E73ED2E0587D
:107B6000F040E0F78ACF823631F489E55CDF80E0CF
:107B70005ADF80E896C0823419F0873609F07DC05C
:107B8000332443DFD82F41DFC82F3FDF082F835432
:107B9000843008F085C0063411F4440C551CF20101
:107BA00010926F001736B9F4033489F483E09DDC3A
:107BB000AEDC8EB51EBC37DF0DB42197D1F7A4DC47
:107BC00008C0063411F4859101C03FDC2CDF2197F9
:107BD000C2F72F014AC00334A9F4E11104C081DCCB
:107BE00088ED83DC8BDC7DDC82E07FDC0EDF0DB496
:107BF0008EBDCA95D9F731968BDC80DCDA9569F7B2
:107C00002F0131C00634F1F49F01F437D8F4E5D1E7
:107C100019C0FBDE063461F4C0FB46F0F43728F4EB
:107C2000182E81E087BFE89511243296082E0AC0ED
:107C3000043439F4DF01B370AD59B94F8D933196E7
:107C400001C007DC21972AF7043431F42F01F370C7
:107C5000FE2B49F466DC07C0063429F42F01F90134
:107C6000F43708F4B8D18DE0DEDE063411F4569412
:107C7000479482E080936F0015C08237E1E049F0BD
:107C80008634E0E031F08E34E3E019F0813531F4F0
:107C9000E2E0F0E089E087BF849103C08B3111F00E
:107CA0008FE3C1DE83E0C1DB55D095FF03C009C07F
:107CB0007ED171F058D080FFFBCF4CD002C077D17D
:107CC00039F051D080FFFBCF84E0AFDB8BE743C0BE
:107CD0000895E4E5F1E067E090915B0180915C013B
:107CE000913231F0913AE1F58132D1F55ED181C026
:107CF000823271F48191805B8191844089F5809119
:107D00005D0180FD2DC0F89481E08093E00078CD86
:107D1000803231F54AD14BD1E9F08530D9F023D00A
:107D200083FD18C082FFF7CF04C07ADE81936150D3
:107D300031F09091F3008091F200892BB1F7C6DF0A
:107D4000611549F704C033D129F0853019F00BD003
:107D500080FFF9CF8EE79091E80089238093E800B7
:107D6000089584E062DB8091E80008958091E2004C
:107D70000895FCDF8E7F80618093E200089582E0A9
:107D800061EC09D083E061E802D084E060E842E180
:107D900003C080E060E042E048DB81E007D0109261
:107DA000ED006093EC004093ED0008959091EB009E
:107DB000892B8093EB00089560E0923029F0913098
:107DC00029F4E0E062E102C0E2E16EE3F1E008954F
:107DD00080915B0188234CF402C0E9D0C1F3C3DF7A
:107DE00082FFFBCF73CFE3D091F3BDDF80FFFBCFEA
:107DF000B1CF40916101509162014617510520F0C9
:107E0000462F611509F4A6DF50E022C0D0D061F101
:107E1000853051F1A8DF83FD59CFA5DF82FD21C058
:107E200080FF16C03091F3002091F20006C08191CE
:107E30008093F10041502F5F3F4F411519F02830DA
:107E40003105A8F350E02830310509F451E082DF14
:107E50004115E1F65523D1F604C0A9D029F08530AB
:107E600019F081DF82FFF9CF31CFEBE5F1E0D8DD0A
:107E70008193E336E1F72DDF76DF83FF91C08091B8
:107E80005B0190915C01913009F170F09330F1F059
:107E9000953009F444C0963009F456C0983009F47E
:107EA00060C0993059F767C0823841F780915F010F
:107EB000BBDA2091EB001092E90077D0229526954D
:107EC00021702093F1001092F10052C0882311F02C
:107ED0008230A1F68F71823089F680915D0188230E
:107EE000D1F420915F01277049F22093E90080913D
:107EF000EB0080FF10C0933011F480E20BC080E1F2
:107F000055DF81E0880F2A95E9F78093EA00109207
:107F1000EA0088E04BDF1092E90047D02AC08823AE
:107F200091F410915D0110680FB7F8943ED050DFC6
:107F30001ADF80FFFDCF1093E300103883E009F4CF
:107F400082E08EBB0FBF2CC08058823048F58091F4
:107F50005D0190915E0130DF603011F126D049DF84
:107F60001FC08038E9F421D0809153018093F10043
:107F7000F1DE2EDF15C0882399F490915D019230D7
:107F800078F49093530111D023DF8091530188231B
:107F900021F48091E30091E087FD94E09EBBEFDE49
:107FA000E2DE83FF089580E201DF87EFD4CE8EB357
:107FB00088230895A3E6B1E0F437B8F40ED090E436
:107FC0000D901D9081E087BFE89532969A95C1F794
:107FD0001124E058F04085E001C083E001D081E148
:0C7FE00087BFE89507B600FCFDCF0895B0
:067FFA003139DDCFFBDC94
:040000030000740085
:00000001FF
